:020000040000FA
:10000000850186018316A22AFE00FE0E030E8301DF
:10001000D5000408D6008C1CA5288C10BD0B132815
:100020003230BD00BC17C6082F1C031919288615CD
:100030001A2886110B302906031D28282808203E7F
:100040008400000EF0397D1CF0300606F03986067B
:100050002B308400FB20031C840A00080A3C29067C
:10006000031D3728F03006040606F03986060230F4
:100070002906031D3D28F8308605A90B4B280B30B7
:10008000A900A80A2808063A0319A800280A0606A3
:1000900007397D188606AE0F5728AD0F5728AF0ACF
:1000A0007D15AB202F185728C608031DC603CF188F
:1000B0009C28CF1D6128D00B9C28851ACF11D00A0F
:1000C0009C284F1C6B28851A9C284F10D1010430A6
:1000D000D20006308C2805084F06203903197628EF
:1000E000CF064F1602304F1B0630D0004F1B83281F
:1000F000D00B9C280310851A0314D20DD10D4F1775
:100100004F1204308C284F1A8E28D00B9C284F0891
:1001100082390938CF008030D0009C284F13D11F7E
:100120009C28D20DD10D520DD10DD213511FD217D3
:10013000D11A0314D20CCF14051CC2030518C20A2D
:10014000C10BA5286430C100CC2356088400550E8D
:1001500083007E0E09003C30AE00F630AD00080092
:10016000F101F10AF63E0318B1280A3EF103F10E3F
:10017000710708002F3084007830E4203C30E42000
:100180001830E4202030B6003308F000B319F00A2C
:10019000701CB603023A031DD228B6033408033993
:1001A000031DB6033608E4200318B20A0D30E4201C
:1001B0000318B30A6430E420643035020318B50133
:1001C0007D114F1D0800092D000203188000840ACC
:1001D0000318800A0800D32431080006F000840ABE
:1001E00030080006840A7004031DF8284708C6007A
:1001F000F10BEC28080048083102031C0800310A02
:10020000490208003108F43E031C310803190C3E72
:1002100008000F30A000A100A200A300A400A500C8
:10022000FD10FD1B2F1C15290800FC199029013019
:100230008A007C08073982077829722967294E29A4
:100240003B2942294829352951081F39D21B323E02
:1002500088210530A2005208802900305B18013047
:100260005D210430A200590853292B0A5D21033077
:10027000A2002C0A532909307D1BA00043089E21AF
:100280004408532948085D210130A2004908532938
:100290000230A2007D0E0339A5000800370A5D2157
:1002A0001830FD190C30B020F0000F39A500700E89
:1002B0000F3903190F30A4000800B020F0000F39E7
:1002C000A100700E0F3903190F30A0000800350887
:1002D00088213408B020F0000F39A300700E0F39C8
:1002E000A20008003408882133086A2132088029D6
:1002F0003108FD1902215D2130086A2103102F0CFD
:10030000B020F0000F39A500700E0F39A4000800CE
:10031000B020F0000F39A100700E0F39A0000800C6
:100320007C080739013EA000FB21183000060319A4
:10033000080000089E21840A00088029B020F000EF
:100340000F39A300700E0F3903190F30A2000800F7
:10035000510854061F39D41B0039031D5D2A520869
:10036000D30603195D2A7F39F0004030F1000130D7
:100370008A0071087225F10AF200F11EF21B5D2A53
:100380007006031DB92971031F398207112A0C2A2F
:10039000142A1A2A202A252A2B2A302A362A3B2ACE
:1003A000412A522A452A502A4A2A002A052A022A84
:1003B000E629EF295D2A5D2A5D2A5D2A5D2A5D2AEC
:1003C0005D2A5D2A5D2A5D2A5D2A5D2AF921FC19D4
:1003D000AE2B03308A007C0D0E399E3E8200F9213F
:1003E000840AFC19C32B03308A007C0D0E39B13E00
:1003F00082000A30AA007C0D0E39A03E840008005D
:10040000C6015D2A0130FD065D2A0A30AA007C0A79
:100410007C060F39FC065D2AAF0AAF0A78302F023E
:100420000318AF01AB20582A0230AF027830031C0A
:10043000AF07122AB00A3C3030060319B000582A20
:10044000B003B01F582A3B301E2AB10A18303106BB
:100450000319B100582AB103B11F582A1730292AAD
:10046000360332060319B201B20A532AB20B532AD9
:100470003603B200532A0C3033060319B300B30A13
:10048000532AB30B532A0B303E2AB4036330B41FF4
:10049000532AB400B5036330B51BB5000230542AAB
:1004A000B50A4E2AB40A0130FC000A30AA005A2AC2
:1004B000FC01AA01FD134F157D155908DA005208F9
:1004C000D300CF100800183A031D183A452D041028
:1004D00018300006041403198000FD1404100408E9
:1004E0007F39F80019307722840A3C30772A0002DD
:1004F000031880000008452D7E229D2BFD14153029
:10050000F80048086322C80049086322C9000800AF
:100510008A229D2BFD141730F8000730AB05AC057F
:100520002B0845252C08452D98229D2B9C229D2B80
:100530007D077D063039FD061430F8007D087839D6
:10054000FD14452D8601F93092008C14831207307A
:100550009F008301203084008001840A841FAC2A1C
:100560000508D800C503C2176430C1004016023028
:10057000A9003E3072253F390319013EC7003F30C4
:100580007225D4004F148B247D1405309200FD1485
:100590008C01C0308B00CF18A82140083639203A92
:1005A00003195E247D1D042BBA207D25B700FD14A0
:1005B0002F18DF2AAA08031DAA0BDF2AFC01FC085A
:1005C000031DEB2A3C302F067D1B031DEB2A0A304E
:1005D000AA000130FC00AF08031D042B45083006BB
:1005E0000319F42AC506EB203008031D042B430829
:1005F000C400C301FB20C6080318031D042B0130EF
:10060000FD1A02217D1AC600FD180921BC1F9D2B71
:10061000BC13031085180314B80D380903191C2BDB
:10062000C03A32300319BA003808FE3A031D232BB2
:100630003C1E202B3C12232BBA0B232B3C16FC1701
:100640003C143230BA00031085190314B90D39096E
:100650000319362BC03A32300319BB003908FE3A71
:10066000031D3D2BBC1E3A2BBC123D2BBB0B3D2B5F
:10067000BC16FC17BC143230BB003C0830390319DF
:10068000FC133C1C6C2B3C10C6010A30AA003C1A1F
:100690004C2B0130FD066C2B7D1C492BF921FC19DC
:1006A000662B03308A007C0D0E398207B10A692B54
:1006B000B30A692BB50A692BFD11962A7D13962A78
:1006C000C80A7C2AF030942AAB0A882A800A6D2254
:1006D0006C2BFD137D154F15BC1C9D2BBC10C6014A
:1006E0000A30AA00BC1A7C2B7D1C7A2B7C0A7C0663
:1006F0000F39FC067D149D2B7D1C7A2BF921840A71
:10070000FC19972B03308A007C0D0E398207B00A42
:100710009A2BB20A9A2BB40A9A2BFD15962A7D17AA
:10072000962AC90A7C2A1030942AAC0A882A800AA0
:1007300067229D2BFD137D154F15CB2A00005D2AE6
:1007400000005D2A00005D2AFD11C62B7D13C62B1B
:10075000C80AC82BF030CA2BAB0AC12B800A6D2205
:100760005D2A00005D2A00005D2A00005D2AFD155B
:10077000C62B7D17C62BC90AC82B1030CA2BAC0A52
:10078000C12B8A225D2A800A67225D2A9C225D2A6B
:100790007E225D2A98225D2ABF0A03194D2C03018F
:1007A000C21B0130C201C2174006013903190800FB
:1007B000C006401EEB2B4018F22BB5303F07031C40
:1007C000E42BE73E031CE62BC0120800E130C00515
:1007D000BE01BE03ED2B4018F42BE2303F07031C93
:1007E0004D2CBE0ABF010800F1303F0703184D2C05
:1007F000F9303F07031CFE2BC017032CFD303F07C9
:10080000031C4D2CC013BF01C0124E3084003A307F
:100810003E0203193F2C083E0318362C8001840346
:10082000083E0318362C80018403063E0318362C3C
:1008300080018403013E03183F2C063E0318362C2A
:1008400080018403013E03183F2C073E0318362C19
:100850008001013E03183C2C033E031D0800C01814
:100860000800C01B4017C01F40130800400D800C3B
:100870000830C01BC0060800C01F4D2C08000830FF
:10088000C01BC006C0194C2C3A303E060319C018D4
:100890000800C30AC0164E2C4015C01440160800AC
:1008A0008403000CF000700C3F39F3000F39731A09
:1008B0000A3EF31A143E731B283E08004E30840093
:1008C000000855243406F100B4068403000CF0003F
:1008D000F00C700C1F3955243306F104B306502474
:1008E0003206F104B20650243106F104B106840345
:1008F000000C7F3955243006F104B00603102F0C8C
:10090000F104AF01C012AB20F108031908007D15F6
:100910004F15FD130800AF0101302B25B03EAF0D80
:10092000AB202C255524AF07AF072C255524B0004C
:100930002C255424B1002C255424B200FA0EFA0CB4
:100940007A0C0339F2002C251F395524B3001030DE
:100950002B25B4002C25FF3A3406031DDA2C2C2558
:10096000B5002C252C257D067839FD062C25C800E0
:100970002C25C9002C25AB002C25AC002C25DB0038
:100980002C25D900D3242C258000840A2C25800016
:10099000840AF10BC32C34087206033903190800CA
:1009A000B40ABA20202D2030F800A030840008308E
:1009B000F10008000C30B100B001AF010130B2000D
:1009C000B701B300B4001430B5001330F8000030A4
:1009D000FC0045258030FD00783945250830C800E9
:1009E00045251430C90045250730AB004525AC002E
:1009F0004525030145255A304525D324183080006C
:100A00004525840A003080004525840AF10BFE2C20
:100A100008008030292503012F18503E44252F0C53
:100A2000442530084425310844253208B0203418C4
:100A30004038B418803845253308442528254F11FF
:100A40001030F80034084525340945253508452D72
:100A50000030F801452DF800502556255525502524
:100A6000A13056254E25F3156C2583120310051A67
:100A700003148316FA0D6A25F30B342D61254C25DA
:100A8000F80A7A0883120800B020FA00502556258B
:100A900055257A0856253F2D63256C2505166D2DA5
:100AA00083164E256C2563256A2D7808FB000830D7
:100AB000F300FB1B4E25FB1F63256525FB0DF30B88
:100AC000592D4E25652505126D2D05150930F900A6
:100AD000F90B682D05116D2D05150830F900F90B7E
:100AE0006F2DA034831603139B00831603131C146D
:100AF000831603131A0883010800F001F101F201C3
:100B00003208F3003408F600F7013508F400031941
:100B10008F2D6430F6070318F70AF40B892D0310A4
:100B20003308FD3EF400F41F982D0C30F4078317B2
:100B3000F8257307F200831FA12DF603760A031927
:100B4000F703770CF400760CF3006D30F2070130F8
:100B5000FD25F1070318F00AF60BA52DF703F71F83
:100B6000A52D1F30F2074330FD25F1071A30FD2572
:100B7000F007F40CF30C3508831FC12DB4080319DA
:100B8000FF3EF600F302031CF403F60C760C3F392B
:100B900073070318F40AF2077408FD25F107031818
:100BA000F00A8301F501F3010730FB00F601F701BC
:100BB0002030F400F30DF20DF10DF00DF60DF70DF0
:100BC000F40D7508F6027B08031C7B0A77020318F4
:100BD00074147418EE2D7508F6077708F7000310E3
:100BE000F40CF40BDA2DF30DF20DF10DF00D0800FD
:100BF00007308A007408F23E82000318013E0800A4
:0C0FE40000341F343D345C347A349934FE
:100FF000B834D634F534E23EE23E543EF10A0800FD
:084000000900010001000800A5
:02400E00423F2F
:1042000036002000740075006200650020004E003A
:104210006900780069006500200063006C006F0091
:1042200063006B00200077006900740068002000C4
:104230004400430046003700370020007300790037
:104240006E006300680072006F006E002000610065
:104250006E0064002000490032004300200052003C
:0442600054004300C3
:04427C000800160020
:104280000000100011001A001B001C001D0012008D
:1042900013001400150027001F004D004E000D00F4
:0A42A0006C006B006D006E008000E2
:00000001FF
